:10000000F4C1189518951895189518953EC287C291
:040010001895189592
:1000280000002A2000002D2000002A202D2000009A
:100038002D202A2000202D202A2020202D202D2090
:100048002A202D20202020202D202A202D202A2063
:1000580020202D202D202A202D20202020202D205A
:100068002A202D202A2020202D202D202A202D2036
:10007800202020202D202A202A2020202A2020204D
:1000880020202D202A202D000A140A0A140A1414EC
:0A0098000A00727633646F732D00C6
:1003E80033C0F8942FE52DBF22E02EBF2FEF27BB97
:1003F80020EF28BBA5D02FEF28BB22272BBF22E850
:1004080029BF24E023BF25E02EBDD19AA098A1984A
:10041800A298A398A89AA99AAA9AAB9A29E1209394
:10042800610020E02093640022ED209362002FEF0A
:1004380020936300209162002DBD209163002CBDA4
:10044800F0E0E8E311277894112309F006D00000C2
:100458000000000000000000F7CF9A9B05C00000D4
:100468009B9B05C0000009C0F0E0EAE203C0F0E091
:10047800EEE200C025E02EBDC5CD0895F0E0E2EA29
:1004880008952F933F934FB6C895002DE3950030FC
:1004980039F422272093640020E02EBD1FEF37C0D7
:1004A8000A3249F42FEF209364002DEF2DBD2FEF72
:1004B8002CBD11272CC0003249F422272093640058
:1004C8002DEF2DBD2FEF2CBD112721C00D3249F482
:1004D8002FEF2093640029EF2DBD2FEF2CBD11279E
:1004E80016C00A3049F42FEF2093640022E62DBD90
:1004F80023E62CBD11270BC0043149F42227209391
:1005080064002AEF2DBD2FEF2CBD112700C04FBE70
:100518003F912F9118952F933F935FB620916400D8
:100528002F3F09F009C02BB332E023272BBB2091C2
:1005380061003FEF321B32BF5FBE3F912F9118958C
:1005480004E61AEF24E82A95F1F718941A95D1F7DA
:0A05580018940A95B1F7189408955D
:00000001FF
